:100000000C9438000C9453000C9453000C9453003F
:100010000C947E040C9453000C9453000C945300E5
:100020000C9453000C94E3030C9453000C94530071
:100030000C9453000C9453000C9453000C945300F4
:100040000C940F040C9453000C9453000C943F0731
:100050000C94390E0C9453000C9453000C945300E0
:100060000C9453000C9453000C9453000C945300C4
:1000700011241FBECFEFD4E0DEBFCDBF12E0A0E061
:10008000B1E0EAE0F9E302C005900D92A436B107B1
:10009000D9F713E0A4E6B2E001C01D92A63EB10775
:1000A000E1F70C940F060C94000090919002292F18
:1000B000221F2227221F892F82958695869583707D
:1000C0002827892F82958F702827892F86958695D6
:1000D00028272170892F9927880F991F282B209373
:1000E0009002822F99270895FF920F931F93F894FF
:1000F000809166028150823000F1809171028630D9
:1001000010F0109271028091710280FF02C09498E9
:1001100004C0949A88EF0E9423088091710288237A
:1001200039F0809171028F5F80937102789447C398
:10013000809171028F5F809371028091650280FFD0
:10014000E4C18091BB0299278830910541F1893043
:10015000910594F48330910509F48AC084309105A7
:100160001CF4019721F10AC38530910509F41EC1E1
:10017000079709F4A1C002C38B30910509F49CC014
:100180008C30910524F4099709F410C1F7C28D3021
:10019000910509F40BC10F9709F48EC0EFC280E0FE
:1001A0000E94770F80918B020E94E408E7C2809141
:1001B0007103882321F480916603882361F0909174
:1001C0008B029F3F41F0991F9927991F80918702C9
:1001D000892B0E94770F80916603882309F4CEC291
:1001E00080916E03803150F480916E03E82FFF27D9
:1001F000EC58FC4F80818F3F09F0C0C210926E0313
:1002000080916D038F5F80936D0380916D038031CA
:1002100068F480916D03E82FFF27EE0FFF1FEA5B64
:10022000FC4F808191818F5F9F4F11F410926D037D
:1002300080916D03E82FFF27EE0FFF1FEA5BFC4F55
:100240008081918190936903809368038091680312
:10025000909169038F5F9F4F21F48FEF8093740318
:100260008DC20E940311809381020E94E70B86C217
:1002700080917103882309F481C280918B028F3FA2
:1002800029F0881F8827881F0E94770F80916E03AE
:100290008F5F80936E0380916E03803150F4809164
:1002A0006E03E82FFF27EC58FC4F80818F3F09F049
:1002B00065C210926E0362C28091C503882309F45F
:1002C0005DC290918B029F3F41F0991F9927991F22
:1002D00080918702892B0E94770F20918B02822FB9
:1002E00099278F739070892B21F080918102820F62
:1002F00001C0822F0E94E40880916E03803150F487
:1003000080916E03E82FFF27EC58FC4F80818F3FD0
:1003100009F034C210926E038091C4038F5F809302
:10032000C4038091C403803248F48091C403E82F51
:10033000FF27EC55FC4F80818F3F11F41092C403CE
:1003400064EA73E084E893E00E94D018882331F0D7
:1003500090918502809184029817A1F0A4E8B3E0FF
:10036000E4EAF3E09FE18D918193915097FFFBCFF9
:100370001092C40310928102109280020E94100D0C
:100380000E94B90D80918402809385028091800241
:10039000809381028091C403E82FFF27EC55FC4F26
:1003A0006081809185020E944A15E8C18091C50351
:1003B000882309F4E3C190918B029F3F41F0991F7C
:1003C0009927991F80918702892B0E94770F20918E
:1003D0008B02822F99278F739070892B59F010917F
:1003E0008102120F80916803909169030E94EE10C0
:1003F000810F01C0822F0E94E40880916E0380313A
:1004000050F480916E03E82FFF27EC58FC4F808159
:100410008F3F09F0B3C110926E0380916D0380315C
:1004200070F480916D03E82FFF27EE0FFF1FEA5B4A
:10043000FC4F808191818F5F9F4F09F050C01092D7
:100440006D038091C4038F5F8093C4038091C403C4
:10045000803248F48091C403E82FFF27EC55FC4F0D
:1004600080818F3F59F51092C40364EA73E084E8F9
:1004700093E00E94D018882331F0909185028091FA
:100480008402981791F0A4E8B3E0E4EAF3E09FE176
:100490008D918193915097FFFBCF10928102109222
:1004A00080020E94100D0E94B90D809184028093F9
:1004B0008502809180028093810205C08091C403EF
:1004C0008F5F8093C4038091C403E82FFF27EC550E
:1004D000FC4F6081809185020E948F1105C0809140
:1004E0006D038F5F80936D0380916D03E82FFF276D
:1004F000EE0FFF1FEA5BFC4F8081918190936903AF
:10050000809368030E94031139C18091BB0299272F
:100510008830910541F18930910594F4833091053B
:1005200009F48EC0843091051CF4019771F126C145
:100530008530910509F4BFC0079709F4B2C01EC108
:100540008B30910509F4ADC08C30910524F40997E6
:1005500009F4B1C013C18D30910509F4ACC00F97F7
:1005600009F49FC00BC180918B028093640280913B
:100570008A0280938B020E94550080938A028091A8
:100580008B0240E0642F8F73F3C080917103882346
:1005900029F480916603882309F4F0C080917103E7
:1005A000882379F080916E03803148F480916E0346
:1005B000E82FFF27EC58FC4F80818F3F11F41092F9
:1005C0006E0360918B026093640280916E03E82F4A
:1005D000FF27EC58FC4F8F5F80936E03E081E09320
:1005E0008B02EF3F09F4CAC080918602882319F07C
:1005F000E07CE0938B0220918B02822F99278F73EE
:100600009070422F4295469546954370661F662727
:10061000661F2F73892B59F0417080918802482BF7
:1006200080918702682B80918102820F37C04170D0
:1006300080918802482B80918702682B822F2EC0E0
:1006400080917103882309F499C00E94E70B80917F
:100650006E030E940B0C80918B0280936402809148
:100660006E03E82FFF27EC58FC4F808180938B02AC
:100670008F3F09F483C00E94500D20918B02922F6E
:100680009295969596959370917080916402881FCB
:100690008827881F492F682F822F8F730E945C0F35
:1006A0006DC08091C503882331F00E94E70B8091D3
:1006B0006E030E940B0C8091C503882309F45EC071
:1006C00000918B020093640280916E03E82FFF2754
:1006D000EC58FC4F8F5F80936E03E081E0938B02B8
:1006E000EF3F09F44BC080918602882319F0E07C2B
:1006F000E0938B0220918B02822F99278F73907049
:10070000422F4295469546954370602F661F662797
:10071000661F2F73892B21F151E0F52EF422809171
:100720008802F82A00918702062B10918102120F8D
:1007300080916803909169030E94EE104F2D602F05
:10074000810F0E945C0F10918B0280918102180F23
:1007500080916803909169030E94EE10810F0CC094
:10076000417080918802482B80918702682B822FEC
:100770000E945C0F80918B020E94C00880916502EC
:10078000843030F485E20E94440B0E94AB0D09C016
:1007900080916502883028F485E20E94A60B0E94B1
:1007A0009E0D0E948D0D809165028F5F8093650282
:1007B00080916502883010F01092650278941F9144
:1007C0000F91FF9008951F920F920FB60F92112470
:1007D0002F933F934F935F936F937F938F939F9349
:1007E000AF93BF93EF93FF93809191029091920208
:1007F00090938900809388000E947400FF91EF918C
:10080000BF91AF919F918F917F916F915F914F9128
:100810003F912F910F900FBE0F901F9018951F9230
:100820000F920FB60F9211242F933F934F935F9324
:100830006F937F938F939F93AF93BF93CF93EF93D8
:10084000FF93809172028F3F29F0809172028F5F37
:100850008093720280918202909183028F5F9F4FFA
:1008600049F08091820290918302019690938302D5
:100870008093820280916F0290917002892B81F0A7
:1008800080916F0290917002019790937002809313
:100890006F0280916F0290917002892B09F49498F5
:1008A000809166028130C1F4C0B3C295CF70C1702F
:1008B00080916C02882371F4CC2361F080917002E6
:1008C000909171020196909371028093700288EF6B
:1008D0000E942308C0936C02FF91EF91CF91BF91CA
:1008E000AF919F918F917F916F915F914F913F91C8
:1008F0002F910F900FBE0F901F9018951F920F927F
:100900000FB60F9211242F933F938F939F9329B388
:10091000237080919302281791F1833041F42230A3
:1009200099F480918E0290918F02019709C08230D4
:1009300059F4233049F480918E0290918F020196F0
:1009400090938F0280938E0280918E0290918F02FD
:100950008D52914030F08CE291E090938F02809321
:100960008E0280918E0290918F02449730F484E140
:1009700090E090938F0280938E02209393029F9138
:100980008F913F912F910F900FBE0F901F90189550
:1009900043E350E081B1886981B940B920E030E09B
:1009A0002CBF4FE150E08AB188698AB949B920BDAE
:1009B00080EC8ABB8CE38BBB8BEB87BB18BA8FEFC9
:1009C00084BB81BB86B981E58DB9089589B7816003
:1009D00089BF8BE083BF8AEF81BF089580917D003E
:1009E000846080937D00089585E20E94A60B80912B
:1009F0007D008B7F80937D000895E199FECF9FBBA2
:100A00008EBBE09A8DB39927089580917D008695DD
:100A100086959927817090700895E199FECF9FBBCC
:100A20008EBB6DBBF894E29AE19A789408950F9387
:100A30001F93CF93DF938C0181E00D32180710F0E4
:100A40000CE211E00431110510F404E110E0109300
:100A50008D0200938C0210938F0200938E02812FDF
:100A60009927682F85E090E00E940D0560918C0227
:100A700086E090E00E940D0580918C0290918D029D
:100A80000E94FA0DC0E0D0E7E8E3F9E398014427BB
:100A90005527BE01CF010E94631CFA01E90193E0D2
:100AA000F695E795D795C7959A95D1F7BE01CF01F1
:100AB00026E030E040E050E00E94631CFA01E901CA
:100AC000CA01AA27BB279C01009731F4D093920258
:100AD000C093910281E061C0887F892B69F403E0B3
:100AE000F695E795D795C7950A95D1F7D0939202D9
:100AF000C093910282E051C0C901807F892B69F4C3
:100B000014E0F695E795D795C7951A95D1F7D09348
:100B10009202C093910286E040C0C901807E892B79
:100B200069F4B5E0F695E795D795C795BA95D1F7ED
:100B3000D0939202C093910287E02FC0C901807CBC
:100B4000892B69F4A6E0F695E795D795C795AA9500
:100B5000D1F7D0939202C093910283E01EC0C901E5
:100B60008070892B51F48D2F9E2FAF2FBB27909330
:100B700092028093910284E010C020703C7F232B6E
:100B800079F46AE0F695E795D795C7956A95D1F718
:100B9000D0939202C093910285E080938A0002C0B4
:100BA00010928A0080919102909192029095819585
:100BB0009F4F90939202809391029093890080932B
:100BC0008800DF91CF911F910F9108950F931F938C
:100BD00080916B00816080936B0080916B008260DC
:100BE00080936B008BB788608BBF85E090E00E949C
:100BF000FD049927182F002786E090E00E94FD044D
:100C00009927802B912B0E941705109265028091E5
:100C10007D00846080937D001F910F910895CFEF38
:100C2000D4E0DEBFCDBF0E94C8040E94E6050E944A
:100C3000E60480918C02809390020E945E090E94DB
:100C4000910778940E94AA098091BB029927883065
:100C5000910509F453C089309105CCF48330910596
:100C600071F18430910554F48130910569F182303D
:100C700091050CF052C0892BB9F1E4CF8530910574
:100C800059F185309105ACF1079731F1DBCF8C300C
:100C9000910509F442C08D3091051CF40A97E9F1E1
:100CA0001DC08E30910531F08E30910594F00F9774
:100CB00081F0C8CF109266020E94510FC3CF1092EC
:100CC00066020E94FF15BECF109266020E94FC11C0
:100CD000B9CF1092660205C081E001C082E0809326
:100CE00066020E94E918AECF109266020E94350893
:100CF000A9CF109266020E947E0FA4CF10926602C6
:100D00000E94EE040E94D20B0E94AA098091BB02AD
:100D10008830D1F30E94F40495CF0E94D20B0E9438
:100D20008D0D90CF159BFECF83B980E090E00895A4
:100D3000CF93DF93EC018881882331F089910E9461
:100D4000920688818823D1F7DF91CF9108950F9380
:100D50001F93CF93DF93EC0100E117E2CE01B801BE
:100D60000E944F1C6115710581F0862F805D0E94E5
:100D70009206CE01B8010E944F1CEC01C8016AE046
:100D800070E00E944F1C8B010EC0CE01B8010E9482
:100D90004F1CEC01C8016AE070E00E944F1C8B01FF
:100DA0006A307105D8F601151105A9F0CE01B80118
:100DB0000E944F1CCB01805D0E949206CE01B801BB
:100DC0000E944F1CEC01C8016AE070E00E944F1CB9
:100DD0008B01672B59F7DF91CF911F910F910895E8
:100DE0008F708A3010F4805D01C0895C0E94920689
:100DF00008950895CF93DF93EC01892F9927829569
:100E00008F70009711F00E94F0068D2F99270097A0
:100E100011F00E94F006CE0144E0969587954A9520
:100E2000E1F7009711F00E94F0068C2F0E94F00667
:100E3000DF91CF91089582B1992787FD90958827FA
:100E4000990F881F99270895179BFECF83B1992783
:100E5000089520EA3FE0E22FF32F3197F1F78A95CA
:100E6000D1F708958AEF0E9429078AEF0E94290787
:100E70008AEF0E9429078AEF0E94290708951F928E
:100E80000F920FB60F9211248F939F93EF93FF93BE
:100E90009CB1983FB1F480916602813021F0949A20
:100EA00085E080936F028091C503882349F180918A
:100EB000670290916802019690936802809367029E
:100EC0001FC080916A02E82FFF27EB56FD4F9083E9
:100ED0008F5F80936A0280916A028F7180936A02A9
:100EE00090916A0280916B02981751F480916B0285
:100EF0008F5F80936B0280916B028F7180936B0286
:100F0000FF91EF919F918F910F900FBE0F901F90C7
:100F1000189599270E94FD04803108F08FE09927E9
:100F2000089583E00E9489078093B50284E00E94BF
:100F3000890780939402089590916B0280916A02D0
:100F4000981719F081E090E0089580E090E008950E
:100F5000089590916B0280916A029817D1F3F894EA
:100F600080916B02E82FFF27EB56FD4F8F5F809338
:100F70006B02908180916B028F7180936B027894E9
:100F8000892F992708950E949C07892BC1F00E9400
:100F9000A90787FF14C0682F62956F70482F5527E7
:100FA0006F3059F09A012F7030708091B5029927F7
:100FB0002817390721F460936902CA01089580E077
:100FC00090E00895089590916402891741F480E0BB
:100FD0000E94770F0E94220D8FEF80936402089584
:100FE0000895FF920F931F93CF93C82F00E0F02E28
:100FF000662321F4602F0E94E30720C080916402E1
:101000008F3F09F001E0653610F081E0F82E1C2FCB
:1010100019514F2D602F812F0E945C0F812F0E944C
:10102000500D81E0F81619F48F2D0E94440B013009
:1010300019F482E00E94440BC0936402CF911F9187
:101040000F91FF9008955D9BFECF8CB980E090E0FA
:10105000089580919402806B0E9423088BE70E9480
:10106000230880E00E94230808951F93CF930E94D5
:10107000F4040E94E70B8091B5020E940B0C1091C2
:10108000C2028FEF809364020E94AA098091BB0282
:10109000882319F00E94290870C00E943E0B882303
:1010A00039F1412F55278091C202992701969C0161
:1010B000207F3170821B930B2091B502481759078E
:1010C00021F4222339F0215003C02F3019F02F5F73
:1010D0002093B5026091B50283E090E00E940D0577
:1010E0000E94E70B8091B5020E940B0C1091C20286
:1010F0000E949C07892B41F20E94A907482F582F74
:10110000551F5527551FA1F0682F62956F706F30DE
:1011100049F099278F7090702091B502332782177C
:10112000930719F46093690203C010926902ACCF6F
:101130008091690299278830910589F0099709F013
:10114000A3CF552321F00E94A907C82F01C0C42FA7
:101150000E94A907682F8C2F0E94F10795CF552375
:1011600021F00E94A907C82F01C0C42F0E94A9071F
:10117000682F8C2F0E94E30787CFCF911F9108958E
:10118000CF93C82F8091940280690E9423088C2FEE
:1011900099278F739070892B11F480E003C08C2FF6
:1011A0008F73875E0E9423088C2F82958695869583
:1011B000837080FF03C08091020102C08091000112
:1011C0000E942308CF910895CF93C82F8091940255
:1011D00080680E9423088C2F99278F739070892B29
:1011E00011F480E003C0CF738C2F875E0E94230828
:1011F000809101010E942308CF9108958091660299
:10120000823029F08CEF0E9423080E94290808955B
:101210000895CF930E940505C82F80916602813002
:10122000D1F0CC2311F00E94F4049498979A85E0B1
:101230000E94290780919102909192020A979093BF
:101240008900809388001092710210926502CC236D
:1012500011F00E94EE04CF910895809166028130D2
:1012600009F097980895089590B3991F9927991FA9
:1012700080916E02882339F4992329F090936E02AD
:1012800081E090E0089590936E0280E090E00895F0
:10129000089590B3991F9927991F80916D02882313
:1012A00039F0992329F490936D0281E090E008953C
:1012B00090936D0280E090E00895089581B3806F6F
:1012C00081BB82B38F7082BB08958FE091B3982366
:1012D00091BB92B3982392BB0895DE980895AC0118
:1012E000F894C0980000000000000000C09A20E0C0
:1012F0001FB8779BFECFFA01E20FF11D8FB18083FB
:101300002F5F2330A8F37894089599B39695969516
:101310009F70292F269526952695892F8695827070
:10132000282B892F9927880F991F382F3470232B4A
:10133000880F991F880F991F8870282B8FE0821BB8
:1013400099270895DE9A089589B3869586958F70BA
:1013500099270895AF92BF92CF92DF92EF92FF92BA
:101360000F931F93CF93DF93CDB7DEB726970FB6BA
:10137000F894DEBF0FBECDBF20918E0230918F0258
:1013800080918C0290918D022817390731F080915D
:101390008E0290918F020E941705AFEBB2E0E8EB4E
:1013A000F2E042E011921D92415047FFFBCF809145
:1013B0007202843108F490C0109272020E946D098A
:1013C000CE0101960E946F098091BC028C838091AE
:1013D000BD028D838091BE028E8340E001E010E06B
:1013E0005E01A00EB11E842F869586958695A82F46
:1013F000BB27BD0164547D4F842F8770980102C0C4
:10140000220F331F8A95E2F7C901FB013081232F98
:101410002823FD01ED53FD4FE081E823AA0DBB1DFC
:10142000AC91A8234F5F8095222319F03823EA2B33
:1014300002C03823EA233E2BFB013083483198F267
:101440000E948509482F8091C202481749F0809177
:10145000B702481729F44093C20281E080937302D7
:101460004093B7020E94A2096FEBC62E62E0D62E0F
:1014700058EBE52E52E0F52E0CEB12E0BE016C5F4E
:101480007F4FA3ECB2E042E0F50181915F018D93C3
:10149000FB012191BF01F80181918F01922F9827C3
:1014A0008923F70181937F019223F60191936F01C4
:1014B000415047FFE9CF0E94A409482F8091BB0209
:1014C000481731F08091B602481711F44093BB02DF
:1014D0004093B6020E948D0D26960FB6F894DEBF9B
:1014E0000FBECDBFDF91CF911F910F91FF90EF9075
:1014F000DF90CF90BF90AF900895282F883118F0DB
:1015000080E090E00895869586958695E82FFF27E0
:10151000E454FD4F80819927277002C095958795E7
:101520002A95E2F79C012170307080FF03C081E0B2
:1015300090E00895C90108950895282F883118F082
:1015400080E090E00895869586958695E82FFF27A0
:10155000E854FD4F80819927277002C095958795A3
:101560002A95E2F79C012170307080FF03C081E072
:1015700090E00895C90108950895282F883118F042
:1015800080E090E00895869586958695E82FFF2760
:10159000E154FD4F80819927277002C0959587956A
:1015A0002A95E2F79C012170307080FF03C081E032
:1015B00090E00895C901089508958091BC028823A0
:1015C00059F48091BD02882339F48091BE028823AA
:1015D00019F481E090E0089580E090E00895089586
:1015E000FF920F931F93CF93DF93FF2400E010E04F
:1015F000CBE0D1E088810E947D0A882311F0C801E8
:1016000009C0F39421960F5F1F4F8CE08F1594F75C
:101610008FEF9FEFDF91CF911F910F91FF90089572
:10162000CF93C0E0EC2FFF27ED5FFE4F80810E943B
:101630007D0AEC2FEF5F882319F08E2F992705C0C4
:10164000CE2FE83078F380E090E0CF910895CF93EB
:10165000C0E0EC2FFF27ED5FFE4F80810E949D0AC6
:10166000EC2FEF5F882319F08E2F992705C0CE2F1E
:10167000E83078F380E090E0CF9108958091730294
:101680001092730299270895282F883290F4869536
:1016900086958695E82FFF27E758FD4F277081E054
:1016A00090E002C0880F991F2A95E2F72081282B2D
:1016B000208308950895282F883290F48695869582
:1016C0008695E82FFF27EC58FD4F277081E090E0CA
:1016D00002C0880F991F2A95E2F72081282B2083CA
:1016E00008950895282F8832A0F4869586958695CA
:1016F000E82FFF27EC58FD4F277081E090E002C0F3
:10170000880F991F2A95E2F7982F90958081892359
:10171000808308950895282F883218F080E090E0A3
:101720000895869586958695E82FFF27EC58FD4FFE
:10173000277081E090E002C0880F991F2A95E2F798
:1017400020812823822F992708950895282F8832F1
:10175000A0F4869586958695E82FFF27E758FD4FDC
:10176000277081E090E002C0880F991F2A95E2F768
:10177000982F909580818923808308950895282F3C
:10178000869586958695E9E7F2E0E80FF11D808160
:101790009927277002C0959587952A95E2F7817061
:1017A0009070089510927D0210927C0210927B023C
:1017B00010927A02109279021092780210927702B7
:1017C00010927602109275021092740208950F938F
:1017D0001F93CF9305E411E0CFE0F80181918F01D1
:1017E0000E94A60BC150C7FFF8CFCF911F910F9158
:1017F00008950F931F93CF9305E411E0CFE0F80114
:1018000081918F010E94720BC150C7FFF8CFCF9119
:101810001F910F910895803138F4E82FFF27EB5B7B
:10182000FE4F80810E94440B08950895803138F462
:10183000E82FFF27EB5BFE4F80810E945B0B089532
:101840000895803118F020E030E009C0E82FFF272C
:10185000EB5BFE4F80810E94BF0B282F3327C9010D
:101860000895803118F080E090E00895E82FFF2778
:10187000EB5BFE4F80810E948B0B992708950895A2
:10188000883138F4E82FFF27E35DFE4F80810E9406
:10189000440B08950895883138F4E82FFF27E35D5D
:1018A000FE4F80810E945B0B08950895883138F4C3
:1018B000E82FFF27E35DFE4F80810E94A60B08956D
:1018C00008950F931F93CF930DE211E0C7E1F80144
:1018D00081918F010E94A60BC150C7FFF8CFCF9115
:1018E0001F910F910895E82F8150883030F4FF2721
:1018F000EC5DFE4F80810E94440B089508951F9374
:10190000CF93182F81E0E82FFF27C82FCF5F8117D3
:1019100031F4EC5DFE4F80810E94440B05C0EC5D0C
:10192000FE4F80810E94A60B8C2FC93060F3CF91AF
:101930001F910895E82F8150883030F4FF27EC5D27
:10194000FE4F80810E94A60B08950895E82F8150D4
:10195000883030F4FF27EC5DFE4F80810E94720BCF
:1019600008950895E82F8150883030F4FF27EC5D0A
:10197000FE4F80810E945B0B08950895E82F8150EF
:10198000883040F4FF27EC5DFE4F80810E948B0B76
:101990009927089580E090E008950895E82F8150F8
:1019A000883048F4FF27EC5DFE4F80810E94BF0B1A
:1019B000282F332702C020E030E0C90108950F939B
:1019C0001F93CF9305E211E0C7E0F80181918F01E9
:1019D0000E94A60BC150C7FFF8CFCF911F910F9166
:1019E00008958D3038F4E82FFF27E85EFE4F8081A0
:1019F0000E94440B089508958D3038F4E82FFF2796
:101A0000E85EFE4F80810E945B0B08950895E8E137
:101A1000F1E0E80FF11D80810E948B0B992708955A
:101A20000F931F93CF9308E111E0CCE0F80181916F
:101A30008F010E94A60BC150C7FFF8CFCF911F9115
:101A40000F9108950E94100D84E00E94A60B83E080
:101A50000E94A60B88E00E94A60B81E00E94A60BC4
:101A600082E00E94A60B0895CF93C82F84E00E94C5
:101A7000A60BC23021F483E00E945B0B0FC083E011
:101A80000E94A60B83E00E94720BC13011F483E028
:101A900003C0CF3F19F484E00E94440BCF91089516
:101AA000CF93C82F0E94220DC7FF03C086E10E947A
:101AB000400C8C2F829586958695837080FF03C09D
:101AC00085E10E94400CCF7311F48C2F15C0C731F3
:101AD00010F48FEF11C0C43218F4CC5080E00CC069
:101AE000C03318F4C85181E007C0CC3318F4C45295
:101AF00082E002C083E0C0530E94340DCC2321F465
:101B000084E10E94400C07C0EC2FFF27E35FFE4FEB
:101B100080810E94440BCF910895F894DF98E9E703
:101B2000F2E080818FB9779BFECF319682E0ED376E
:101B3000F807B9F3B4F3DF9A78940895A4E7B2E014
:101B4000E9E7F2E024E080819D91892B8193215087
:101B500027FFF9CF0895A4E7B2E0E9E7F2E024E037
:101B60009D919095808189238193215027FFF8CF03
:101B70000895A4E7B2E0E9E7F2E034E020819C9127
:101B8000822F892319F09095292320831D923150AB
:101B9000319637FFF3CF0895AC0120E0322F611565
:101BA000710581F0FA01E30FF11D80812827E22FF2
:101BB000FF27EB5AFE4F20813F5F832F992786171F
:101BC000970780F3822F992708950F931F93CF9340
:101BD000DF936115710549F08C01EB01F8018191EA
:101BE0008F010E9492062197C9F7DF91CF911F9133
:101BF0000F9108950F931F939C0106EC12E082E46D
:101C00008093C6021092C70282E08093C802832F9D
:101C100099278093C9022093CA0265E070E0C80149
:101C20000E94CC0D8093CB0266E070E0C8010E9458
:101C3000E50D1F910F9108950F931F9306EC12E08D
:101C400090E89093C6021092C70291E09093C80268
:101C50008093C90264E070E0C8010E94CC0D8093BB
:101C6000CA0265E070E0C8010E94E50D1F910F9166
:101C700008951F920F920FB60F921124EF92FF92C8
:101C80001F932F933F934F935F936F937F938F9304
:101C90009F93AF93BF93CF93DF93EF93FF9393B152
:101CA00080915502882309F4E4C080917F0280343A
:101CB00048F4E82FFF27EA5FFC4F90838F5F809303
:101CC0007F0204C00E941C0E10927F0220917F02AE
:101CD000233008F4CEC0F090060380910703682FEC
:101CE0007727762F6627809108039927682B792B11
:101CF0003327CB0104962817390708F4BAC0FB0133
:101D0000EA5FFC4F1381EB012396BE0186E093E06E
:101D10000E94CC0D181791F0BE0186E093E00E945E
:101D2000CC0D99270E94FA0610927F0280E00E9453
:101D30001C0E0E94E70B0E948D0D9DC08F2D9927D0
:101D40008131910551F18231910544F48130910541
:101D500009F488C0409709F460C086C080349105BA
:101D600021F08134910541F07FC080918C029091E7
:101D70008D020E94FA0D7BC080910803823009F029
:101D800073C0809109039927982F882720910A030F
:101D9000820F911D0E9417056AC08091080382304E
:101DA00009F062C08091090390910A03C82FDD27D2
:101DB00063E0CC0FDD1F6A95E1F7C90FD11D89E102
:101DC0008093C6021092C70280E18093C8020F2E52
:101DD000F9ECEF2EF2E0FF2EF02DC295D295D07FD8
:101DE000DC27C07FDC271FE0CE010E94AB10F7018B
:101DF00081937F011150219617FFF6CF63E170E0C8
:101E000086EC92E00E94CC0D8093D90264E170E0F0
:101E100086EC92E00E94E50D2AC080910803823191
:101E200019F58091090390910A03C82FDD2733E04B
:101E3000CC0FDD1F3A95E1F7C90FD11D2BE0E22E43
:101E400023E0F22E94E0CC0FDD1F9A95E1F71FE01E
:101E5000BE01F70181917F010E946C101150219603
:101E600017FFF6CF81E001C080E00E941C0E1092A7
:101E70007F020E94E70BFF91EF91DF91CF91BF911D
:101E8000AF919F918F917F916F915F914F913F9112
:101E90002F911F91FF90EF900F900FBE0F901F900A
:101EA00018950E94AA098091BB028E30D1F30E943E
:101EB000D20B0E948D0D089590E03A98803408F07E
:101EC0008FE3611160E4442311F440E801C0492F1D
:101ED000882349F0862B842B85BB3A9A9F5F9832E2
:101EE000E8F3399A0895642B65BB08950895882313
:101EF00011F0AE9A01C039983A9808957F928F9266
:101F00009F92AF92BF92CF92DF92EF92FF920F9388
:101F10001F93CF93DF93EE24FF248824982C0E94F4
:101F2000EE040E94E70B7090C202670157010E9405
:101F3000AA098091BB02843019F00E942908BEC012
:101F4000809194020E94210C882331F40E94E70BB7
:101F5000809194020E940B0C0E943E0B882309F191
:101F6000472D55278091C202992701969C01207F19
:101F70003170821B930B209194024817590721F46A
:101F8000222339F0215003C02F3019F02F5F209306
:101F900094026091940284E090E00E940D0570909C
:101FA000C2028E2D0E94340D992019F081E00E940A
:101FB000440B882019F082E00E94440B00E0C6E543
:101FC000D2E088810E949D0A8823B9F0102F1A0D53
:101FD000195E492D682D812F0E945C0F892D99274C
:101FE00056E0880F991F5A95E1F7812B0E94C0088F
:101FF000812F0E94500D41E0842E88810E94BD0AED
:10200000882379F0202F2C0D295E892D992736E021
:10201000880F991F3A95E1F7822B0E94E4080E94ED
:10202000220D0F5F21960D3060F28FE00E949D0A15
:10203000882351F082E0E816F104D4F40894E11CFE
:10204000F11C8CE090E010C08EE00E949D0A882375
:1020500079F09FEFE9169FEFF90651F04CF00894E4
:10206000E108F10884EF9FEFA80EB91EC80ED91E33
:1020700085E10E949D0A882371F080E0992009F48F
:1020800081E0982E882321F081E00E94440B03C058
:1020900081E00E94A60B83B399278F739070892BE0
:1020A00009F445CF0E94DD0A882309F440CF80E07F
:1020B0000E94770F0E94220D882439CFDF91CF91A3
:1020C0001F910F91FF90EF90DF90CF90BF90AF9056
:1020D0009F908F907F900895282FF89495E0C09856
:1020E00000000000000000009FB9779BFECF0000B9
:1020F0000000000000001FB8779BFECF8FB1C09A90
:10210000000000000000000080FDE9CFC098000042
:10211000000086E08FB9779BFECF00000000C09AD8
:102120000000000000000000C0980000000082E0F5
:102130008FB9779BFECF872F99278FB9779BFECFDB
:102140006FB9779BFECF2FB9779BFECF00000000C1
:10215000C09A789408959C01F894C09800000000FB
:1021600083E08FB9779BFECF832F99278FB9779B19
:10217000FECF2FB9779BFECF000000001FB8779BE2
:10218000FECF8FB1C09A78949927089510926A0370
:10219000109271031092660380E00E94770F0E94F4
:1021A000D20B0E94B90D0E943E0B089510926B0352
:1021B00084E20E94A60B0E94D20B0E94B90D1092DD
:1021C000710380E00E94770F089581E080936B0394
:1021D00084E20E94440B0E94E70B0895892F9927FF
:1021E000282F2F71822F992787FD909534E096959F
:1021F00087953A95E1F7892B09F0206E822F992770
:1022000087FD909508952091680327708091680359
:1022100090916903F3E096958795FA95E1F7622F1F
:102220008F700E944A1560916803709169039B0149
:1022300044275527DA01C90180709078A070B070EA
:10224000892F9A2FAB2FBB2780938602DA01C90111
:1022500080709074A070B070892F9A2FAB2FBB271D
:10226000809388022070307240705070BB27A52F79
:10227000942F832F8093870210926E03CB010E94CC
:10228000EE109927089581E080936A0381E20E940D
:10229000440B10928802809188028093870280917B
:1022A00087028093860210926603109271038091D8
:1022B00046039091470390936903809368038F5F6F
:1022C0009F4F89F010926D0310926E0310928B0253
:1022D0000E940311809381028091650280FDFCCFF2
:1022E00081E0809366030E94E70B0895809181024C
:1022F000882321F483E00E94A60B0CC087FF07C04F
:1023000083E00E94A60B84E00E94440B089583E0C2
:102310000E94440B84E00E94A60B08950895FF924A
:102320000F931F93CF93DF93C82FDD2703E0CC0FCC
:10233000DD1F0A95E1F7C60FD11D15E0CC0FDD1F9B
:102340001A95E1F7BFE0FB2EC050D84F06E413E02A
:10235000CE010E94AB109927982F8827F80180831F
:102360009183CE0101960E94AB10282F3327F801EC
:1023700080819181822B932B819391938F01FA9489
:102380002296F7FEE5CFDF91CF911F910F91FF903D
:102390000895FF920F931F93CF93DF93C82FDD27EC
:1023A00053E0CC0FDD1F5A95E1F7C60FD11D45E074
:1023B000CC0FDD1F4A95E1F73FE0F32E06E413E072
:1023C000C050D84FF80180819181892F9927BE0193
:1023D0000E946C102196F801819191918F01BE01AC
:1023E0000E946C10FA942196F7FEECCFDF91CF910A
:1023F0001F910F91FF9008951F93CF93DF930E9439
:10240000EE048091C20287708093670310926C0380
:1024100010926B0310926A0310926603109271037C
:1024200010926D038FEF9FEF909369038093680381
:10243000109266020E94E70B0E94B90D0E94AA0941
:102440008091BB02813071F00E94F40410927103FC
:102450001092660380E00E94770F0E94D20B0E94C8
:102460008D0DEEC280916B03882361F580916A0324
:10247000882341F50E943E0B882359F08091C202C7
:1024800087708093670360916C030E948F110E9494
:10249000E70B809167030E940B0C0E94100BC82F62
:1024A000882359F00E94100D8C2F815080936C036B
:1024B000682F809167030E948F1180916C038F5F5A
:1024C0000E94730C81E00E949D0A882379F080911C
:1024D0006A03882319F00E94C61008C080916B031C
:1024E000882311F00E94D6100E94431180916A0344
:1024F000882329F480916B03882309F463C08091B9
:102500006D030E94310C882311F40E94B90D809153
:102510006D030E94160C80916803909169038F5F90
:102520009F4F21F40E94220D80E046C080E00E946F
:10253000A60B809168039091690343E09695879577
:102540004A95E1F78F700E940B0C8091680390917F
:10255000690397FF04C088E00E94440B03C088E031
:102560000E94A60B8091680390916903AA27BB275C
:102570003EE0B695A795979587953A95D1F78170E6
:102580009070892B21F081E00E94440B03C081E010
:102590000E94A60B8091680390916903AA27BB272C
:1025A0002DE0B695A795979587952A95D1F78170D7
:1025B0009070892B21F082E00E94440B03C082E0DE
:1025C0000E94A60B88E00E949D0A882331F483E0D4
:1025D0000E949D0A882309F478C010916A03112390
:1025E00009F073C0812F0E94770FC0916B03CC2339
:1025F00009F442C088E00E949D0A8823D1F08091AE
:102600006D039927019640976CF480916D03E82F34
:10261000FF27EE0FFF1FEA5BFC4F808191818F5FE8
:102620009F4F19F410936D0330C080916D038F5F3D
:1026300020C080916D038823C9F480916D03992790
:102640000196409714F580916D03E82FFF27EE0F58
:10265000FF1FEA5BFC4F808191818F5F9F4FA9F044
:1026600080916D038F5F80936D03E7CF80916D0341
:10267000815080936D0309C088E00E949D0A8823E1
:1026800021F00E94E510C0936D0380916D03E82F47
:10269000FF27EE0FFF1FEA5BFC4F80819181909333
:1026A000690380936803109271038F5F9F4F69F0F5
:1026B0000E9403118093810210926E038091650243
:1026C00080FDFCCF81E08093710387E10E949D0A29
:1026D000882339F180916B038823E9F080916D03A1
:1026E00099270196409764F480916D03E82FFF27A6
:1026F000EE0FFF1FEA5BFC4F8FEF9FEF8283938308
:102700008FEF9FEF90936903809368030E94D61028
:1027100080E00E94A60B60916C03809167030E9489
:10272000C91180916B03882309F47CC180916803EF
:10273000909169038F5F9F4F09F40FC184E10E945C
:102740009D0A882311F180916D03E82FFF27EE0F7A
:10275000FF1FEA5BFC4F8081918120E030E88227F7
:1027600093278083918380819181909369038093E3
:102770006803AA27BB2780709078A070B070892F5B
:102780009A2FAB2FBB278093860285E10E949D0A7A
:10279000882311F180916D03E82FFF27EE0FFF1FB3
:1027A000EA5BFC4F8081918120E030E4822793270F
:1027B00080839183808191819093690380936803E2
:1027C000AA27BB2780709074A070B070892F9A2FB1
:1027D000AB2FBB278093880286E10E949D0A882345
:1027E00011F180916D03E82FFF27EE0FFF1FEA5BC9
:1027F000FC4F8081918120E030E282279327808303
:102800009183808191819093690380936803AA27C3
:10281000BB2780709072A070B070892F9A2FAB2F59
:10282000BB27809387028FE00E947D0A882331F4C2
:102830008EE00E947D0A882309F47DC00E94F00A80
:10284000C82FDD27C7FDD0958FE00E949D0A882301
:1028500029F48EE00E949D0A882351F00E94B90D50
:102860000E94100D83E00E94A60B84E00E94A60B3C
:102870008FE00E947D0A882349F183E00E94440B87
:102880008FEFCF3FD807C9F00E94B90D20916803A0
:1028900030916903307E9C2F8827282B392B309369
:1028A00069032093680380916D03E82FFF27EE0FE3
:1028B000FF1FEA5BFC4F2083318380916803909176
:1028C00069030E94EE108093810232C08EE00E9464
:1028D0007D0A882309F441C084E00E94440B2FEF55
:1028E000CF3FD207E1F00E94B90D209168033091EB
:1028F0006903307E2C97CF71D0709C2F8827282BAE
:10290000392B309369032093680380916D03E82F7E
:10291000FF27EE0FFF1FEA5BFC4F2083318380917E
:102920006803909169030E94EE1080938102845F96
:102930000E94FC0C12C08FE00E94BD0A882329F47B
:102940008EE00E94BD0A882341F083E00E94A60B1E
:1029500084E00E94A60B0E94B90D8FE00E947D0AC0
:10296000882309F05FC08EE00E947D0A882309F069
:1029700059C00E94270BC82F882329F40E943E0BC0
:10298000882309F447C00E94DF0C0E94E70BCC2388
:1029900059F480916803909169038F5F9F4F29F0EC
:1029A000C0916803C77001C0C1501092710380E0EC
:1029B0000E94770F4091C202242F332763E0220F39
:1029C000331F6A95E1F78C2F9927282B392B3093E9
:1029D00069032093680380916D03E82FFF27EE0FB2
:1029E000FF1FEA5BFC4F208331836C2F842F0E94F2
:1029F0004A1510926E03109287028091870280938D
:102A0000880280918802809386021092810281E080
:102A1000809371030E9476118091680387708F5FA5
:102A20000E947F0C80916A03882309F407CD0E94DD
:102A300076118091680387708F5F0E947F0CFECCB7
:102A4000DF91CF911F91089510926E0381E08093E2
:102A50006F0381E20E94440B80E00E94770F0E9486
:102A6000EE048091650280FDFCCF81E080937103CC
:102A7000089581E080936B0384E20E94440B0E94DE
:102A8000E70B80E00E940B0C0E94F40480E00E949F
:102A9000770F0895EF92FF920F931F93CF93DF93D9
:102AA000182F062F0E948D0DC12FDD2723E0CC0F9C
:102AB000DD1F2A95E1F7C00FD11D94E0CC0FDD1F7B
:102AC0009A95E1F784E7E82E83E0F82E1FE0CE0127
:102AD0000E94AB10F70181937F011150219617FFDF
:102AE000F6CF809174038F3F41F487E1E4E7F3E090
:102AF0001FE08193115017FFFCCF0E948D0DDF91D5
:102B0000CF911F910F91FF90EF900895EF92FF9258
:102B10000F931F93CF93DF93182F062F0E948D0DD5
:102B2000C12FDD2753E0CC0FDD1F5A95E1F7C00F11
:102B3000D11D44E7E42E43E0F42E34E0CC0FDD1F3A
:102B40003A95E1F71FE0BE01F70181917F010E94F4
:102B50006C101150219617FFF6CF0E948D0DDF915A
:102B6000CF911F910F91FF90EF90089510926B03FA
:102B700084E20E94A60B0E94610C0E94E70B8091E8
:102B8000C2020E940B0C0E94EE0480E00E94770FAC
:102B900008950E94F404109271030E94610C0E9437
:102BA000E70B8091C2020E940B0C10926F0381E22E
:102BB0000E94A60B80E00E94770F089581E0809329
:102BC00073030E94EE0480E00E94770F0E94610C64
:102BD00080E00E945B0B8091C2020E940B0C8091EE
:102BE00070038F5F0E94730C08951092730380E04E
:102BF0000E94720B0E94610C0E94E70B0895EF92F5
:102C0000FF920F931F93CF93DF9310927003109254
:102C10006B0310926F031092730310927103109262
:102C20006E0310928B02109266020E94AA09809194
:102C3000C20280937203609170030E944A150E9441
:102C4000D20B8091C2020E940B0C0E94EE040E94E3
:102C5000AA098091BB02833081F00E94F404109293
:102C6000710380E00E94770F0E942D090E94FE08E8
:102C70000E94D20B0E948D0D8CC2909172038091A4
:102C8000C2029817F9F080916F03882311F00E9417
:102C9000C91580916B03882311F00E94B61590919D
:102CA000C2029093720380917303882329F4609188
:102CB0007003892F0E944A150E94E70B8091C2027F
:102CC0000E940B0C80916F038823F9F480916B03B1
:102CD0008823D9F4809170038F5F0E94730C0E9447
:102CE000100BC82F882389F00E94100D8C2F0E9492
:102CF000730C6C2F61506093700380917303882371
:102D000021F4809172030E944A1580E00E949D0A7E
:102D1000882399F080916F03882379F082E20E94E2
:102D2000440B04E713E0CFE00E945500F8018193C3
:102D30008F01C150C7FFF8CF0CC080E00E94BD0AD0
:102D4000882339F080916F03882319F082E20E9472
:102D5000A60B81E00E949D0A8823A9F0809173034D
:102D6000882311F00E94F51580916F03882319F0D4
:102D70000E94C91508C080916B03882311F00E943E
:102D8000B6150E94241580916F03882329F4809141
:102D90006B03882309F427C100916E03E02EFF2402
:102DA000E701CC58DC4F18811F7385E10E949D0A12
:102DB000882331F01F3321F0888190E489278883AC
:102DC00086E10E949D0A882349F01F3339F0F701FC
:102DD000EC58FC4F808190E8892780831F3341F0B5
:102DE000112331F0173110F4CFEF0DC0143210F46D
:102DF000C0E009C0103310F4C1E005C01C3310F46A
:102E0000C2E001C0C3E084E10E949D0A811110E08C
:102E10008FE00E949D0A882339F01F3329F0112387
:102E200019F01C160CF0145F8EE00E949D0A882396
:102E300041F01F3331F0112321F0CF3F11F00CF09E
:102E40001C5084E00E949D0A882331F08CE0C80267
:102E5000C0011124182F195E89E00E949D0A882361
:102E600031F08CE0C802C0011124182F185E85E0F3
:102E70000E949D0A882331F08CE0C802C001112411
:102E8000182F175E8AE00E949D0A882331F08CE09B
:102E9000C802C0011124182F165EC3300CF063C0A5
:102EA00086E00E949D0A882331F08CE0C802C001B0
:102EB0001124182F155E87E00E949D0A882331F0A7
:102EC0008CE0C802C0011124182F145E8BE00E9410
:102ED0009D0A882331F08CE0C802C0011124182F0C
:102EE000135E81E10E949D0A882331F08CE0C802C4
:102EF000C0011124182F125E8CE00E949D0A8823C5
:102F000031F08CE0C802C0011124182F115E82E15B
:102F10000E949D0A882331F08CE0C802C001112470
:102F2000182F105E8DE00E949D0A882331F08CE0FE
:102F3000C802C0011124182F1F5D80E10E949D0A64
:102F4000882331F08CE0C802C0011124182F1E5DC7
:102F500083E10E949D0A882331F08CE0C802C00101
:102F60001124182F1D5D202F3327F901EC58FC4F39
:102F700080818F3F11F41F3319F48081807C182BDE
:102F8000E901CC58DC4F88811817F9F080916B0368
:102F9000882331F080E00E94770F81E00E942907AA
:102FA000188380916B03882381F0812F8295869509
:102FB000869583708170912F991F9927991F482FAB
:102FC000692F812F8F730E945C0F1F3F39F0812F73
:102FD0000E94500D80E00E94A60B05C00E94220DA9
:102FE00080E00E94440B88E00E949D0A882331F40F
:102FF00083E00E949D0A882309F49BC080916B03A3
:10300000882309F46AC080E00E94770F81E00E9463
:10301000290788E00E949D0A8823B1F080916E0301
:103020009927019640974CF480916E03E82FFF2773
:10303000EC58FC4F80818F3F19F410926E0320C032
:1030400080916E038F5F1AC080916E03882399F47C
:1030500080916E038F30A0F480916E03E82FFF27DC
:10306000EC58FC4F80818F3F59F080916E038F5F49
:1030700080936E03EDCF80916E03815080936E0339
:103080000E94E70B80916E030E940B0C80916E03EF
:10309000E82FFF27EC58FC4F808180938B028F3FF5
:1030A00051F481E00E94A60B82E00E94A60B80E012
:1030B0000E94440B3EC080E00E94A60B80918B02D0
:1030C000982F92959695969593709170282F221F20
:1030D0002227221F492F622F25C088E00E949D0AC7
:1030E000882339F1C0916F03CC2319F50E9439155B
:1030F000C0936E0380916E03E82FFF27EC58FC4FBE
:10310000E081E0938B02EF3FA1F08E2F82958695B0
:103110008695837081709E2F991F9927991F482F3C
:10312000692F8E2F8F730E945C0F80918B020E94FB
:10313000500D87E10E949D0A882309F488CD809173
:103140006B03882381F080916E0399270196409745
:1031500044F480916E03E82FFF27EC58FC4F8FEF6B
:1031600081830E94B61580916F03882311F00E941D
:10317000C91580917303882349F060917003809191
:10318000C2020E9486150E94F51561CD0E94DE15CF
:103190005ECDDF91CF911F910F91FF90EF90089539
:1031A00040E0DB01FC0190818C91981719F080E0E0
:1031B00090E0089580818F3F19F481E090E00895B8
:1031C0004F5F31961196403270F381E090E00895A0
:1031D0000895EF92FF920F931F93CF93FF24E090F7
:1031E000BB0280916602882319F40E94EE040BC092
:1031F0000E94F40480916602813019F40E946509EE
:1032000002C00E945E090E94D20B0E94B90D10926A
:10321000A4038091A403809384038FEF8093A5037C
:103220008091A5038093850381E00E94730C109226
:10323000C50310926D0310926E03109269031092F1
:1032400068031092C40310928002109281020E94BF
:10325000E70B8091BB028F3021F08B3011F087306B
:10326000D1F48091C2021AC01092C5030E942D09A8
:103270000E94FE0810928002109281021092870232
:1032800010928602109288020E94D20B0E94B90D01
:103290000E948D0DFEC28091C202877080938502CC
:1032A000809384028091C2020E940B0C0E94AA09A2
:1032B0008091BB028E15C1F687E10E949D0A88238A
:1032C00029F1809182029091830286509D40D0F432
:1032D00080918202909183028E54914098F02091C7
:1032E00082023091830280E69AEEB9010E944F1C5F
:1032F0007093830260938202809182029091830294
:103300000E941705109283021092820280E00E94B0
:103310009D0A882349F00E94100D0E94B90D82E297
:103320000E94440B1092890280E00E94BD0A88230B
:1033300029F1A6ECB3E0E4E8F3E0CFE18D918193CD
:10334000C150C7FFFBCF8091C5038823A1F4A4E837
:10335000B3E0E4EAF3E0CFE18D918193C150C7FF80
:10336000FBCF809180028093810283E00E94A60BB4
:1033700084E00E94A60B82E20E94A60B80E00E94DD
:103380007D0A882361F1C0E080918902C81760F44A
:10339000EC2FFF27EA53FC4F8081883028F48F5FA1
:1033A0000E94730CCF5FF0CF0E94270BC82F882399
:1033B00009F44EC180918902803208F049C1E82F9A
:1033C000FF27EA53FC4FC150C0838F5F809389026F
:1033D000E82FFF27EA53FC4F8FEF808339C18FE03E
:1033E0000E947D0A882331F48EE00E947D0A8823A2
:1033F00009F46DC00E94F00AC82F8FE00E949D0A58
:10340000882329F48EE00E949D0A882339F00E94C7
:10341000100D0E94B90D82E20E94A60B8FE00E945F
:103420007D0A882301F184E00E94A60B83E00E94BC
:10343000440BCF3F11F0C09380028091810287FD41
:103440000AC00E94070D882331F40E94B90D8091B3
:1034500081020E94FC0C9091800280918102981759
:1034600061F1892F28C08EE00E947D0A882329F10E
:1034700083E00E94A60B84E00E94440BCF3F19F02A
:10348000CC50C093800280918102181664F0845F52
:103490000E94070D882339F40E94B90D80918102A2
:1034A000845F0E94FC0C90918002809181029817A9
:1034B00021F0892F845F0E94F10C8091C50388233D
:1034C00009F0C6C08091800280938102C1C08FE064
:1034D0000E94BD0A882329F48EE00E94BD0A882339
:1034E00021F00E94100D0E94B90D0E94100BC82FF0
:1034F000882331F40E943E0B882309F446C01FC084
:103500000E94DF0CC150C093840380918403809398
:10351000C6038FEF80938503809185038093C70353
:103520008091C503882319F5A4E8B3E0E4EAF3E049
:10353000CFE18D918193C150C7FFFBCF18C080911F
:10354000BB028F3021F08B3011F0873019F480915D
:10355000C20203C08091C20287708093840280916E
:10356000C503882321F48091840280938502809191
:10357000C503882351F40E94E70B809184020E94C6
:103580000B0C809180028093810264EA73E084E8EE
:1035900093E00E94D0188823F9F4809185038F3F2F
:1035A00049F48091A5038F3F29F48091A4038F5F94
:1035B0000E94B20CC0E004E813E0F8018081893079
:1035C00008F044C0D8018D918D018F5F0E94730C6B
:1035D000CF5FC03290F33AC0C0E004EA13E0F801D4
:1035E0008081893098F58091C5038823E1F080912E
:1035F000C403E82FFF27EC55FC4FD8019C91808134
:10360000981789F48C918F5F0E94BE0C8823C9F4AF
:10361000F80180818F5F0E949A0CD8018C918F5F96
:103620000E94B20C0EC0F80180818F5F0E94BE0C18
:10363000882311F00E94B90DD8018C918F5F0E94F0
:10364000730CCF5F0F5F1F4FC03248F20E9476119C
:103650008091C503882351F180916602823089F4FC
:10366000809167029091680218161906FCF4809107
:1036700067029091680203979093680280936702B3
:1036800012C0813099F480917002909171021816E5
:10369000190664F4809170029091710203979093DF
:1036A0007102809370020E94740000CE80916602C5
:1036B000823019F40E94C307F82E80916602882395
:1036C00049F481E00E949D0A882321F08091C5037E
:1036D000882371F480916602823021F4BCEFFB16DE
:1036E00039F02BC0813049F50E944909882329F11E
:1036F0001092C50380E00E94770F0E94FE0880911F
:103700006602813011F00E942D0981E20E94A60B11
:103710000E94B90D0E94E70B8091BB028F3021F00F
:103720008B3011F0873019F48091C20203C0809170
:10373000C20287700E940B0C68C0809166028823C9
:1037400049F481E00E949D0A882321F08091C503FD
:10375000882389F080916602823029F48F2D8A5F58
:10376000823048F052C0813009F04FC00E943409C5
:10377000882309F44AC081E20E94440B8091BB0275
:103780008F3021F08B3011F0873039F46091A40331
:103790008091C2020E944A1511C08091C2026091BC
:1037A000A40387700E948F11809146039091470374
:1037B00090936903809368030E94031110928B0217
:1037C00080916602823019F4EBEFFE1631F0109210
:1037D000C40310926E0310926D0310926502109252
:1037E0006802109267021092710210927102109298
:1037F000700281E08093C5038AEF0E9423088091C4
:103800006602813011F00E94090986E10E949D0A3A
:10381000882389F090E080918702882309F491E061
:1038200090938702992321F082E00E94440B03C009
:1038300082E00E94A60B85E10E949D0A882389F000
:1038400090E080918802882309F491E090938802A7
:10385000992321F081E00E94440B03C081E00E9483
:10386000A60B84E10E949D0A882309F41FCD90E0F5
:1038700080918602882309F491E09093860299232F
:1038800021F088E00E94440B11CD88E00E94A60B35
:103890000DCDCF911F910F91FF90EF900895AA1B2E
:1038A000BB1B51E107C0AA1FBB1FA617B70710F02B
:1038B000A61BB70B881F991F5A95A9F7809590955D
:1038C000BC01CD010895A1E21A2EAA1BBB1BFD016C
:1038D0000DC0AA1FBB1FEE1FFF1FA217B307E407EF
:1038E000F50720F0A21BB30BE40BF50B661F771F47
:1038F000881F991F1A9469F7609570958095909527
:0A3900009B01AC01BD01CF01089549
:10390A0064207F04050607111210130409050A062C
:10391A00070B110C120D1013201B191C1A180F0C6F
:10392A000E0B0D0A0920191A180C0B0A0922212557
:10393A002320191A18241B1C0F0E0D04030A0C0B42
:10394A00090801020026271D1E1F10121113141543
:10395A00161705060700070E091C1B1215383F36F5
:10396A003124232A2D70777E796C6B6265484F4625
:10397A004154535A5DE0E7EEE9FCFBF2F5D8DFD695
:10398A00D1C4C3CACD90979E998C8B8285A8AFA6C5
:10399A00A1B4B3BABDC7C0C9CEDBDCD5D2FFF8F13A
:1039AA00F6E3E4EDEAB7B0B9BEABACA5A28F888165
:1039BA008693949D9A2720292E3B3C35321F181155
:1039CA001603040D0A5750595E4B4C45426F686105
:1039DA006673747D7A898E878095929B9CB1B6BFF7
:1039EA00B8ADAAA3A4F9FEF7F0E5E2EBECC1C6CFA5
:1039FA00C8DDDAD3D4696E676075727B7C51565F15
:103A0A00584D4A4344191E171005020B0C21262F44
:103A1A00283D3A33344E49404752555C5B767178BB
:103A2A007F6A6D64633E39303722252C2B060108E4
:103A3A000F1A1D1413AEA9A0A7B2B5BCBB969198D4
:103A4A009F8A8D8483DED9D0D7C2C5CCCBE6E1E884
:103A5A00EFFAFDF4F3010409050A06070B110C122B
:043A6A000D10130028
:00000001FF
